:03000000020100FA
:03000B000203B23B
:03001300020411D3
:10010000758131750932750A32751D00750D0075DE
:100110001C20D210C290C211D212D214D213758CEC
:1001200038758A38758BFD758DFD75880075892247
:1001300075B80275A800D28E12035612041F12035E
:100140008C12036C120471D2AFD2A9D28C12021697
:1001500070AE12033712017F120397E51D6012B4CF
:100160000103020179B4020302017BB403E402013A
:100170007D1201B712032E80D980D780D580D3128B
:10018000035D5002F50822C20C120787C0E0C0824E
:10019000C083C0D07480120719900450751F00C22C
:1001A0000DC20E1207E1D0D0D083D082D0E0E51D81
:1001B00012037E12034022E5086012B46806750837
:1001C000000201D5B46D327508000201E830122931
:1001D000208210C212E50B120352B42401E4F50B85
:1001E00012020F208313C212E50C120352B46001F5
:1001F000E4F50C1201FA12020F22C2A9750D007566
:100200000932750A32758A38D210C28DD2A92212EB
:10021000024912023322D290120457701312048A38
:10022000700E1201FA852C0B852B0CD21412041CB3
:10023000C29022900000780BE61205E91202F3A3A7
:1002400008E61205E91202F322740D120364780B1A
:10025000E612037E120349743A12036408E612039D
:100260007E120349743A12036408E612037E1203F5
:100270004922C0E0C0D0C0F0D20BC0E0C082C08331
:10028000C0D07480120719900441751F00C20DC2BE
:100290000E1207E1D0D0D083D082D0E0748612074E
:1002A00019E50B12037E120340743A120768E50C3D
:1002B00012037E120340E51C120768E50D12037E4F
:1002C000120340D0F0D0D0D0E022900000120636C9
:1002D0001202F3B423030202DC4001E4780BF6A31C
:1002E0001206361202F3B459030202EF4001E47819
:1002F0000CF622400122C0E0C20C120787C0E0C009
:1003000082C083C0D07480120719900426751F0024
:10031000C20DC20E1207E1D0D0D083D082D0E074DB
:10032000C9120719D0E012037E12034080FE301379
:0903300005120249C2132230112A
:1003390005120233C21122120768E5F0120768227A
:10034900120364E5F0120364222401D42243878056
:1003590043985622E599A298C298223099FDC299EC
:10036900F59922900817E493F520900818E493F57D
:100379002112078722F5F0540F4430C5F0C4540FF9
:10038900443022740D120364740A12036422E508CE
:100399006016B42013750800E51D120352B411014B
:1003A900E4F51D600312018722C0E0C0D012049E4B
:1003B900301D0AC21D1201FAD21412041CD50943B8
:1003C900750932D50A3D750A32D212B210201006CB
:1003D900751C20020407751C3AD213E50D1203524D
:1003E900B46019E50C120352B4600CE50B12035208
:1003F900B42401E4F50BE4F50CD211E4F50DD214A3
:1004090012041CD0D0D0E032301405C2141202728A
:10041900D2B332C2B322D2B3C28AD2AA224545503C
:10042900524F4D204143434553530D4641494C5585
:10043900524520282020290054696D653A20004141
:0E0449006C61726D3A20004D6F6465202300D7
:10045700120471D21A12058C3017F8C21A4008D24A
:10046700191204BDC21922020558752532753100CB
:10047700C219C21AC21BC21CC21DD215D218D2166B
:10048700C217221205A430170B1205A4201705E581
:1004970031700122740822201605D52602D216D5FE
:1004A7002513752532201505D52402D215201805E8
:1004B700D52702D2182278287A007B0012058C20D3
:1004C70017055006020555020558EB0B9005E093FA
:1004D7001205683017030205581204F0700AE5F098
:1004E700F608E531B43AE3E422A931B90703020576
:1004F70051B90E03020551B9140630E551020551F1
:10050700B91C0820D010547F020551B9230B20D005
:1005170005543F02055102055BB9290612055E0223
:100527000551B92C0612055E020551B931061205AF
:100537005E020551B9391A12055E12058C20171192
:10054700C5F0EA3330D00502055BF5F0E42274010B
:1005570022740422740222A2D0C0E0EA33FAD0E067
:1005670022F5F0C0F0E412058C301703D0F0221307
:10057700D5F0F3D0F0C0E07408C395F0F5F0D0E003
:1005870003D5F0FC22C0E01205A420170D75240F37
:10059700C2153015FD1205D2921BD0E022752764D3
:1005A700C2181205D220182040F8752764C2181205
:1005B70005D220181350F8C21D05313017077531C1
:1005C70000D21DC217D21C22D21722A2874008755B
:1005D7002605C2163016FDB32207070608070603CD
:0205E700050805
:1005E900C0E01206DC5005D0E002068812069150E0
:1005F90005D0E002068BD0E01206B0500302068E49
:100609001206E9221206DC40761206914074E612BF
:1006190006B0407108A3E582540F70091206E9D5A6
:10062900F0E7020634D5F0E61206E9C3221206DC29
:10063900404D120691404B1206E91206E3E5835438
:10064900072344A11206B01206C640391206E92250
:100659001206DC402A12069140281206E91206E326
:10066900E58354072344A11206B01206C64016F6C4
:1006790008A3D5F0051206E9C3221206FB80EB7424
:1006890001227402227403227B00E5835407234468
:10069900A01206E31206B050081206E9DBEC0206C6
:1006A900AFE5821206B0227A08C280120717C33357
:1006B9009281D280120717DAF0120708227A08E429
:1006C900C280120717D281D280120717C3A28133C1
:1006D900DAEE22C3A2818280B322C28112071722D5
:1006E900C280C281120717D280120717D28112075E
:1006F9001722C280120717C281D28012071722C29D
:1007090080120717D281D280120717A281220022F4
:02081700740A61
:1007190012077C75A0F012072322C2A3C0E0440F80
:1007290052A0D2A3C2A3D0E0C4440F43A0F052A068
:10073900D2A3C2A32275A0F412074522C0F0C2A316
:10074900D2A3E445A054F0C4C2A343A0F0D2A38528
:10075900A0F0C2A353F0F045F0C4C2A3D0F0221216
:10076900077C75A0F21207232212077C75A0F612E6
:10077900074522C0E012073E20E7FAD0E022C0E098
:10078900300A05743812071975A00CC2A375A02088
:10079900D2A3C2A374075521D2E32323120719E573
:1007A90020D2E3540F120719E520C45402D2E212F1
:1007B900071930030CE520C4540CD2E4120719C2FE
:1007C90003200C077401120719D20C300B077402AD
:1007D900120719C20BD0E022200D06E493A30207E9
:1007E900F4200E05E0A30207F4E608D51F0302086A
:1007F90016B40D0302080A6014B4FE0280DAB40AC2
:0E0809000774C012071980D012076880CB2236
:00000001FF
